:020000040000FA
:100000005028A301A200FF30A207031CA307031C72
:100010004B280330A100E3300F200328A101F43E58
:10002000A000A109FE30031C1828A00703181528FA
:10003000A0076400A10F1528000020181F28201811
:10004000212808000310A00DA10DFF3E031822284F
:1000500020084B280038031DFF300405031DFF3026
:100060004B280404031DFF304B281030A800A101C9
:10007000A001A70CA60C031C43282208A0072308F4
:100080000318230FA107A10CA00CA50CA40CA80B0E
:10009000392824084B2883130313831264000800B3
:1000A0008316051405168515051585148612831209
:1000B0008A114D2A83120313E00194013E3094000B
:1000C0008316031306168614831203138C1108007B
:1000D00083120313FF30E70083120313E70B732827
:1000E0000530AC218C2883160313141A792894192F
:1000F0006C2883120313683084007D2160188C28DB
:1001000060100008E500222160188C28840AD10BB9
:1001100081289321601C90286208CF006010B229CA
:10012000080083120313FF30E70083120313E70B69
:100130009C280530AC21DD2883160313141AA2284D
:10014000941995288312031368308400C9288312F8
:100150000313FF30E70083120313E70BB2280530C7
:10016000AC21DD2883160313141AB8289419AB2880
:1001700083120313683084007D216018DD28000895
:10018000E50022216018DD285708E50022216018CB
:10019000DD287D216018DD280008E5006514222196
:1001A0006018DD280E216018DD28840A66088000AA
:1001B000D10BD2289321601CE1286208CF00601087
:1001C000B229080083120313FF30E70083120313E0
:1001D000E70BED280530AC21092983160313141A07
:1001E000F3289419E62883120313683084007D21D4
:1001F000601809290008E500651422216018092902
:100200000E2160180929840A660880009321601C69
:100210000D296208CF006010B22908000830E700FD
:10022000E601E60D031C6610031866143821E11B75
:100230006614E70B11295108E7006117E70B6113FA
:10024000532100340830E7006113E51B6117532187
:100250006018AC216018B229E50D031C6510031865
:100260006514E70B242938210330E11BAC2100344D
:1002700083160313861483120313E11383160313E7
:10028000061683120313061A46294329861C492998
:10029000E11700000000000000008316031306129F
:1002A000831203130034611F61298316031386141C
:1002B00002308312031386186729601CE200601461
:1002C00067298316031386100000000000008316C0
:1002D0000313061600000000000001308312031310
:1002E000061A732970290000000000000000831620
:1002F00003130612831203130034831603138614A8
:100300000616831203130000000000000130061ED1
:10031000AC218316031386100000000000000612B3
:1003200083120313003483160313861006168312F8
:1003300003130000000000000000000000000000A7
:100340000000061EA1298316031386140430861CA0
:10035000AC2183120313003483120313601CE200E8
:1003600060140034861406168316031386140616CA
:100370008312031300340230D1005308E8008312C3
:10038000031368308400840A5008800068208312B8
:1003900003138A11492A0230D1006030E800831229
:1003A000031368308400840A560880006820831292
:1003B00003138A11492A0330D100831203136830D2
:1003C0008400840A4E088000840A45088000682062
:1003D000831203138A11492A0430D10083120313B4
:1003E00068308400840A4E088000840A4508800032
:1003F000840A440880006820831203138A11492A62
:100400000330D1008312031368308400840A4E083D
:100410008000840A440880006820831203138A1134
:10042000492A0230D1008312031368308400840A01
:10043000440880006820831203138A11492A683017
:10044000D7000330D100A030E800831203136830D6
:100450008400840A57088000840A540880006820B9
:10046000831203138A11492A6930D7000330D1005F
:10047000A030E8008312031368308400840A570810
:100480008000840A580880006820831203138A11B0
:10049000492ACF018A015A200800831670308F0044
:1004A00007309C009B018101831286168A015A2025
:1004B00064008A1105185E2A8A01582A52138A118B
:1004C000E72364008A115218672A8A01582A4608CD
:1004D000C70064008A11051C6F2A8A01692A8A11E3
:1004E000E72364008A115218772A8A01582A46089D
:1004F000C800640047080D3C8A11031D812A8A1137
:10050000FE2B64008A11051C872A8A01812A8A1120
:10051000E7230301521CFF30B8004708093C031DC4
:10052000FF30FF3ABA00380884003A088A012A20CE
:10053000BA00BB0064003A083B048A110319A22ADE
:100540008A11FE2B64008A115218A82A8A01582A9F
:100550004608C90064004708093C8A11031DB32AF4
:1005600052178A11FE2B64004708043C8A11031DB0
:10057000BB2A8A11FE2B64004708073C8A11031D21
:10058000C32A8A11FE2B64004708083C8A11031D08
:10059000CB2A8A11FE2B64008A11051CD12A8A01FC
:1005A000CB2A8A11E7230301521CFF30B800470809
:1005B000053C031DFF30FF3ABA00380884003A08B2
:1005C0008A012A20BA00BB0064003A083B048A1161
:1005D0000319EE2A0130CA008A11FE2B64008A1129
:1005E0005218F42A8A01582A4608CA0064008A115F
:1005F000051CFC2A8A01F62A8A11E7230301521CF2
:10060000FF30B8004708063C031DFF30FF3ABA0030
:10061000380884003A088A012A20BA00BB00640026
:100620003A083B048A110319172B8A11FE2B030188
:10063000521CFF30B8004708053C031DFF30FF3A4D
:10064000BA00380884003A088A012A20BA00BB00A0
:1006500064003A083B048A110319302B8A11FE2BDF
:1006600064008A115218362B8A01582A4608CB009A
:1006700064004708053C8A11031D412B52178A115B
:10068000FE2B64008A11051C472B8A01412B8A111D
:10069000E72364008A1152184F2B8A01582A460812
:1006A000CC0064004708063C8A11031D5A2B5217E0
:1006B0008A11FE2B64008A11051C602B8A015A2BBB
:1006C0008A11E72364008A115218682B8A01582A7C
:1006D0004608CD008A11FE2B051A5215051E52112F
:1006E0008519D215851DD21105195216051D5212F4
:1006F0008518D216851CD2120230D21D0301B80013
:100700000030D21D0301B900003052190130B80782
:100710000318B90A0430521E0301BA000030521EF9
:100720000301BB003808BA0739080318013EBB07AC
:100730000830D21E0301BC000030D21E0301BD00F0
:100740003A083C07C60064004608003C8A11031DB5
:10075000AD2B0D30C6008A11E62B640046080A3C1A
:100760008A11031DB62BC6018A11E62B64004608C8
:100770000B3C8A11031DC02B8030C6008A11E62B6A
:10078000640046080C3C8A11031DCA2B8130C60048
:100790008A11E62B640046080D3C8A11031DD42BF8
:1007A0000A30C6008A11E62B640046080E3C8A1106
:1007B000031DDE2B0B30C6008A11E62B64004608B1
:1007C0000F3C8A11031DE62B0C30C6000800D9012E
:1007D000521464008A110518FB2B0A308A0101208B
:1007E000D90A6400653059028A11031CF92B521092
:1007F00008008A01E92B8A016C230800640047087D
:10080000003C8A11031D5E2C4808803C031DFF300C
:10081000FF3AB8004908803C031DFF30FF3ABA0098
:10082000380884003A088A012A20BA00BB004A0826
:10083000803C031DFF30FF3ABC003A083B048400B3
:100840003C088A012A20BC00BD004B08803C031DE7
:10085000FF30FF3ABE003C083D0484003E088A0198
:100860002A20BE00BF004C08803C031DFF30FF3A29
:10087000C0003E083F04840040088A012A20C000CE
:10088000C1004D08003C031DFF30FF3AC200400884
:100890004104840042088A012A20C200C300640087
:1008A000420843048A1103195C2C86120B30A30002
:1008B000B8308A01022086168A11EA2D64004708A2
:1008C000043C8A11031D822CE030D300FF3048071E
:1008D000B800FF300318013EB9000130A00038080D
:1008E0008A012520D0008A01BB214908D6008A014F
:1008F000CB21D0018A01BB218A01BB218A01BB2106
:100900008A11EA2D64004708053C8A11031DC02C9A
:1009100064008A11521FAC2C0A30A600A7014808B7
:10092000A200A3018A013520B8002508B9003808C3
:100930004907CE000A30A600A7014A08A200A30179
:100940008A013520B8002508B90038084B07C500D2
:100950000130C4008A11BA2C4808CE004908C500ED
:1009600064004A08003C8A11031DB82C0130CA00FB
:100970004A08C4006230E8008A01EC218A11EA2D9D
:1009800064004708063C8A11031DF62C64008A1196
:10099000521FEA2C0A30A600A7014808A200A301B2
:1009A0008A013520B8002508B90038084907CE006B
:1009B0000A30A600A7014A08A200A3018A01352037
:1009C000B8002508B90038084B07C5004C08C4001A
:1009D0008A11F02C4808CE004908C5004A08C40016
:1009E0006430E8008A01EC218A11EA2D640047088E
:1009F000073C8A11031D2D2D4808CE004908C4006C
:100A00006630E8004808053C031DFF30FF3AB80097
:100A10004808063C031DFF30FF3ABA00380884003E
:100A20003A088A013120BA00BB004808023C031D85
:100A3000FF30FF3ABC003A083B0484003C088A01BE
:100A40003120BC00BD0064003C083D048A1103193C
:100A50002B2D8A0100228A11EA2D64004708083CE8
:100A60008A11031D5A2DE230D300FF304807B80029
:100A7000FF300318013EB9000130A00038088A0198
:100A80002520D0008A01BB2164004908013C8A115D
:100A9000031D4E2D0130D4008A114F2DD4018A013F
:100AA0001F22D0018A01BB218A01BB218A01BB21FF
:100AB0008A11EA2D64004708093C8A11031DC02DE4
:100AC0004808C40064008A11521BAC2D640044081D
:100AD000003C8A11031D702D3030C4008A11AA2DEC
:100AE00064004408013C8A11031D7A2D3130C40092
:100AF0008A11AA2D64004408023C8A11031D842D2A
:100B00003230C4008A11AA2D64004408803C8A1146
:100B1000031D8E2D2A30C4008A11AA2D64004408BA
:100B2000813C8A11031D982D2330C4008A11AA2DFF
:100B3000640044080C3C8A11031DA22D4330C400FC
:100B40008A11AA2D640044080D3C8A11031DAA2DA8
:100B50004430C4008A11BA2D4808A600A7010A3003
:100B6000A200A3018A013520B8002508B900380881
:100B70004907C4006830E8008A0111228A11EA2D71
:100B8000640047080D3C8A11031DEA2D64004808E3
:100B9000013C8A11031DD42DCE010230C5008030E6
:100BA000C400D2108A11DA2DCE010130C500803088
:100BB000C400D2146230E8008A01EC216430E800FD
:100BC0008A01EC210030D2180130C4006830E800FE
:100BD0008A01112264008A11051CF02D8A01EA2D78
:040BE0008A01582A04
:02400E00703F01
:00000001FF
